:08000000803102288731FD2F39
:100E5C00163021009700080070302100990098018D
:100E6C0022009601080087314227873187313227CB
:100E7C00873187312E27080022008C018E011B3010
:100E8C0021008C0028308E00083023008E000330A7
:100E9C008C0024008C018E012100951722009D01ED
:100EAC009E010800F601F7010130F8000030F9004E
:100EBC000130F2000030F300F401F50187313927DD
:100ECC00873120000C118C160E1274037504031D4F
:100EDC00722F20000C15742F20000C110C1A822F6D
:100EEC0078037904031D822F74037504031D822F6C
:100EFC00F601F701F801F9018E1E892F0130F60772
:100F0C000030F73D8B2FF601F7017708803AF0009F
:100F1C0080307002031D942F0B307602031C9E2F21
:100F2C0078037904031D9E2F0130F4000030F50086
:100F3C007708803AF00080307002031DA72F0B3029
:100F4C007602031CB52F78087904031DB52FF60122
:100F5C00F701F401F5010130F8000030F9007708D1
:100F6C00803AF00080307002031DBE2F33307602C1
:100F7C00031CCF2F78037904031DCF2FF601F70143
:100F8C00F801F901F401F50120000E168C128E1AED
:100F9C00CD2F78037904031DE52F20008C167403E4
:100FAC007504031DE02F720873040319E02FF2017E
:100FBC00F301E92F0130F2000030F300E92FF201C8
:100FCC00F30120008C12720873040319EF2F0E1218
:100FDC00F02F0E160230F1000430F000BA30890BFD
:100FEC00F52FF00BF52FF10BF52F00326B2F2000A6
:040FFC008731582FB2
:020000040001F9
:04000E00E4FFFFFE0E
:00000001FF
